:1000000019C033C032C031C030C02FC02EC02DC087
:100010002CC02BC02AC034C028C027C026C025C091
:1000200024C023C022C021C020C01FC01EC01DC0CC
:100030001CC01BC011241FBECFEFD4E0DEBFCDBF5C
:1000400011E0A0E0B1E0E2E1F2E002C005900D9223
:10005000AA30B107D9F711E0AAE0B1E001C01D92C2
:10006000A431B107E1F7BBD0D2C0CACF8A3010F0BB
:1000700080E00895E82FF0E0E050FF4F8081089580
:100080001F920F920FB60F9211242F938F939F936D
:10009000EF93FF9380910E0190910F010196909341
:1000A0000F0180930E0180910E0190910F01845FEA
:1000B000914008F44DC010920F0110920E018091F2
:1000C00012018F5F80931201809112018A3008F42F
:1000D0003FC01092120180910A018F5F80930A0144
:1000E00080910A018630A0F110920A0180911101DD
:1000F0008F5F80931101809111018A3048F1109235
:100100001101809113018F5F80931301809113017E
:100110008630F0F01092130180910B018F5F809375
:100120000B0180911001823041F480910B018430E9
:1001300020F010920B011092100180910B018A3077
:1001400038F010920B01809110018F5F80931001A5
:1001500080910C018F5F80930C0180910D01880FBD
:1001600080930D0180910C01843029F410920C01D0
:1001700081E080930D0180910C01813051F081303C
:1001800028F0823049F0833099F409C0E0911201DF
:1001900008C0E0910A0105C0E091110102C0E091A0
:1001A0001301EA3028F4F0E0E050FF4FE08101C095
:1001B000E0E088B1807F88B98BB1E095EBB998B168
:1001C00080910D018F70892B88B9FF91EF919F91DC
:1001D0008F912F910F900FBE0F901F9018958AB19D
:1001E0008FEF8AB987B18F6087B98CE790E09093E1
:1001F000890080938800809181008B6080938100CA
:1002000080916F00826080936F007894FFCFF894A4
:02021000FFCF1E
:0A0212003F036D6753767E237F776C
:00000001FF
